:100000000C942A001895000018950000189500001F
:10001000189500001895000018950000189500002C
:10002000189500001895000018950000189500001C
:10003000189500001895000018950000189500000C
:1000400018950000189500001895000018950000FC
:10005000189500008FE58DBFC8E3E0E24E2E84E0E6
:100060008EBFD4E0F4E05F2EA89584B7082E877F7A
:1000700084BF88E1992781BD91BDEEEFF3E0A0E652
:10008000B0E088278D933197E9F766248FEF81BB25
:100090008FE78093600080E090E0A1E6B0E08D9370
:1000A0009C93A1E6B0E00D911C91073050E015073C
:1000B0001CF011F00C947400A0E6B0E08C918F77E6
:1000C0008C93A0E6B0E08C9182BB8CE291E00E9420
:1000D000880091E0A0E6B0E00E949700A1E6B0E0C1
:1000E0000E9478000C9451000C944800F894FFCFC3
:1000F000ED91FC91EF5FFF4FFC93EE9308953197E4
:10010000F1F70895689462F80895E89462F8089504
:10011000EF93FF93EE27E82BE92B31F0E0EAFFE0C5
:100120003197F1F70197D1F7FF91EF910895903052
:1001300039F08C91869508F480689A95D9F78C935C
:02014000089520
:00000001FF
